:100000000C9400280C9402280C9404280C940628C4
:100010000C9408280C940A280C940C280C940E2894
:100020000C9410280C9412280C9414280C94162864
:100030000C9418280C941A280C941C280C941E2834
:100040000C9420280C9422280C9424280C94262804
:100050000C9428280C942A280C942C280C942E28D4
:100060000C943028FFFFFFFFFFFFFFFFFFFFFFFFA4
:10007000FFFFFFFFFFFFFFFFFFFFFFFFFFFFFFFF90
:10008000FFFFFFFFFFFFFFFFFFFFFFFFFFFFFFFF80
:10009000FFFFFFFFFFFFFFFFFFFFFFFFFFFFFFFF70
:1000A000FFFFFFFFFFFFFFFFFFFFFFFFFFFFFFFF60
:10500000AEC10000E1C10000C5C10000C3C1000085
:10501000C1C10000BFC10000BDC10000BBC1000094
:10502000B9C10000B7C10000B5C10000B3C10000A4
:10503000B1C10000AFC10000ADC10000ABC10000B4
:10504000A9C10000A7C10000A5C10000A3C10000C4
:10505000A1C100009FC100009DC100009BC10000D4
:1050600099C1000097C1000005010906A101750161
:105070009508050719E029E715002501810295012A
:105080007508810395057501050819012905910227
:1050900095017503910395067508150025650507AB
:1050A000190029658100C009022200010100803237
:1050B000090400000103010100092101010001228E
:1050C0003F000705810308000A12011001000000DB
:1050D00008424231E10001010200011A0374006933
:1050E000006E00790055005300420062006F0061BD
:1050F0000072006400520368007400740070003A8B
:10510000002F002F006D00610074007200690078AC
:1051100000730074006F0072006D002E0063006F5A
:10512000006D002F006100760072002F007400698E
:10513000006E00790075007300620062006F00610C
:1051400000720064002F000403090474696E79552D
:105150005342626F617264205265762E3320776904
:1051600074682041546D656761333238500A687441
:1051700074703A2F2F6D617472697873746F726DE9
:105180002E636F6D2F6176722F74696E79757362FD
:10519000626F6172642F0A0A0A506C656173652040
:1051A0006361726520617474616E74696F6E206FE3
:1051B000662074686520494E434F4D504154494222
:1051C000494C495459206F6620726567756C61724D
:1051D0002041546D656761382074696E795553427A
:1051E000626F6172640A6669726D77617265732EAF
:1051F00020416C6C206578616D706C6573206E6504
:10520000656420746F20626520636F6D70696C65E2
:105210006420666F722041546D6567613332385087
:105220002C2031364D487A2E0A0A0A0A496E20632C
:1052300061736520796F7520656E636F7574657233
:105240002070726F626C656D732C206861766520CA
:10525000616E79207175657374696F6E73206F72FA
:1052600020696E20636173650A796F75206A7573B2
:105270007420686176652072656D61726B732C2095
:10528000706C6561736520646F206E6F7420686553
:1052900073697461746520746F20636F6E746163E9
:1052A000743A0A5374657068616E20426165727762
:1052B0006F6C6620202D207374657068616E406D80
:1052C000617472697873746F726D2E636F6D0A6D9D
:1052D000617472697873746F726D40676D782E6453
:1052E000652C206F72207374657068616E2E626128
:1052F0006572776F6C664074752D696C6D656E6153
:10530000752E64650A0A5047502D4B65794944094A
:105310003A20307846423942313244420A46696E78
:105320006765727072696E74093A203232353220C4
:105330004234314520313244462034314144203416
:10534000373646203746333620303834412030391E
:105350003131204642394220313244420A00112480
:105360001FBECFEFD8E0DEBFCDBF11E0A0E0B1E0BF
:10537000E8EBFCE502C005900D92A630B107D9F725
:1053800021E0A6E0B1E001C01D92AA34B207E1F726
:1053900023D290C435CEA82FB92F80E090E041E011
:1053A00050EA609530E009C02D9182279795879546
:1053B00010F084279527305EC8F36F5FA8F3089537
:1053C000EADF8D939D930895CF93CFB7CF93DF936B
:1053D000C3954F9BE9F74F9B0BC04F9B09C04F9B59
:1053E00007C04F9B05C04F9B03C04F9B01C08BC0A4
:1053F0006F93C0912D01DD27CC5CDE4F2F9365E5C7
:105400004F9B03C02F916F91E6CF0F931F934F9344
:1054100020E040E15F9309B1047807FB27F93F934F
:1054200050E03BE039C0147840642F77012F5F5F74
:105430001EC0406819B114782F7752501FC04064C5
:1054400009B12F770478D1F15F5F00C023C04062BB
:1054500019B12F77147891F15F5F00C025C00478EF
:105460001027515012F45D5F0000115027952C3F1A
:1054700019B1C8F614780127015027952C3FC8F6BA
:105480004227499309B1047810274F73115027958B
:105490002C3FA8F64695469519B1147879F0012766
:1054A000015027952C3F98F66B5A60F3315009B1A3
:1054B000B0F600C011E01CBB002719C03B5031956D
:1054C000C31BD04011E01CBB0881033C09F10B3425
:1054D000F9F020912B011981110F1213EDCF4A81A0
:1054E000441F093651F10D3211F0013E29F70093A6
:1054F00032013F915F914F911F910F912F916F91C9
:10550000CCB3C0FD65CFDF91CF91CFBFCF911895C0
:1055100020913201222369F310913001112391F57A
:10552000343092F13093300120932C0110912D01F1
:105530003BE0311B30932D0127C000913001013039
:105540000CF50AE54F7049F43091010134FD1DC09E
:1055500000930101C4E1D1E01CC030911F0134FD72
:1055600014C000931F01C0E2D1E013C0052710E072
:1055700000C000000BB91AC0052710E0221F1DC093
:1055800010E021C04AE502C032ED432FC4E1D0E073
:1055900032E01AB114685F9A0BB11AB954E820E8E6
:1055A00065E320FF05270BB9279517951C3FF0F6FB
:1055B0006695B8F7B1F720FF05270BB92795179522
:1055C0001C3FD0F62795179517FF052700001C3FB5
:1055D0000BB9B0F629913A9519F70B771091310173
:1055E000110FC651D0400BB911F010932B0111E0EF
:1055F0001CBB00681AB11B77402F4B7754E05A95BB
:10560000F1F70BB91AB94BB974CF20911F0124FFE0
:1056100007C02091200138E823272093200103C0F0
:105620002AE520931F01FC01A1E2B1E081918D9355
:1056300081E0A932B807D1F768E081E291E0C0DEED
:105640008CE080931F010895FC0188E0DF011D922A
:105650008A95E9F7089580910201909103010196DE
:10566000C9F085B192E0892785B98091000180FF5A
:1056700002C05B9A01C05B988091000181FF02C06B
:105680005D9A01C05D988091000182FF02C0289A56
:105690000895289808951F93CF93DF93CDB7DEB771
:1056A00060970FB6F894DEBF0FBECDBF182FCE01A6
:1056B0000996CADF103211F48CE244C01A3011F49A
:1056C00088E240C0193011F48BE23CC0812F815632
:1056D0008A3110F41D550DC0812F81548A3120F478
:1056E00082E089871D5305C0812F8153893018F4CA
:1056F00013511B8728C0103311F487E223C01034E4
:1057000021F482E089878FE11DC01A3321F482E001
:10571000898783E317C01C3211F486E313C01F325C
:1057200011F484E50FC01A3211F485E50BC01B3269
:1057300011F487E507C01D3211F486E503C01E325F
:1057400011F487E38B8788E0FE013996DE0111961C
:1057500001900D928A95E1F729813A814B815C8114
:105760006D817E818F81988560960FB6F894DEBF3B
:105770000FBECDBFDF91CF911F910895CF93DF93DF
:10578000CDB7DEB760970FB6F894DEBF0FBECDBFC2
:105790008FEF81DF29873A874B875C876D877E870C
:1057A0008F87988B88E0FE013996DE011196019073
:1057B0000D928A95E1F729813A814B815C816D8157
:1057C0007E818F81988560960FB6F894DEBF0FBEFC
:1057D000CDBFDF91CF910895CF93DF93CDB7DEB7E3
:1057E00060970FB6F894DEBF0FBECDBF2FE088E103
:1057F00090E00FB6F894A895809360000FBE2093B8
:10580000600080916900836080936900E89A8BE46E
:10581000809320018AE580931F01579AA895539A97
:10582000559A209A219A5E9856985E9A2FEF83ECAB
:1058300099E0215080409040E1F700C00000A89519
:1058400057987894A89580913001835087FDEFC0D8
:1058500090912D010CE010E0091B11090C5C1E4F0A
:1058600090912C019D3209F0D1C0883009F0DDC043
:1058700083EC809314018AE58093010110920B015F
:10588000F8018081807661F1803241F5818182303A
:10589000C9F018F4813011F505C0893061F08A3003
:1058A000E9F418C08CE091E090932F0180932E01D1
:1058B000CBDE28E0A0C0F80186819781019771F4C2
:1058C0002FEF91C08AE091E090932F0180932E01F9
:1058D00021E091C0F801838180930A0120E08BC010
:1058E000F801928110921D018181811106C01092F0
:1058F0001E018DE191E022E070C0853019F4909393
:10590000310168C0863009F04FC0F80183818130D1
:1059100041F489EC90E590932F0180932E0122E1D0
:105920003FC0823041F487EA90E590932F01809345
:105930002E0122E235C08330F1F4911108C087E4D2
:1059400091E590932F0180932E0124E029C091309E
:1059500041F485EF90E590932F0180932E0122E58D
:105960001FC09230E1F48BED90E590932F0180936E
:105970002E012AE115C0813241F489EB90E5909324
:105980002F0180932E0129E00BC0823241F488E67A
:1059900090E590932F0180932E012FE301C020E02A
:1059A00080E480930B011DC0883069F0893019F4C0
:1059B000909333010FC08A3049F08B3059F48BE457
:1059C0008093200107C083E391E002C08DE191E064
:1059D00021E003C08DE191E020E090932F018093BE
:1059E0002E012F3F41F4F801808187FD268180E858
:1059F00080930B0108C0F8018781811104C0868162
:105A0000821708F4282F209304010FC080910B0106
:105A100087FF0BC0F801808190910001891719F070
:105A20008093000118DE10920401109230018091E1
:105A3000010184FF43C0809104018F3F09F43EC0FF
:105A4000182F893008F018E0811B809304018091A1
:105A5000140198E8892780931401112319F1E0912A
:105A60002E01F0912F0180910B0186FF0BC0A5E163
:105A7000B1E084918D93319685E191E0810F8A1395
:105A8000F8CF0CC0CF01A5E1B1E0FC012191CF011D
:105A90002D9325E131E0210F2A13F7CFF0932F0149
:105AA000E0932E01612F85E191E08ADC1C5F1C30C0
:105AB00019F08FEF809304011093010184E199B1F3
:105AC000947831F48150D9F71092310110922B0162
:105AD00080911F0184FFACC080910201909103016D
:105AE0000196C1F5C0900601D0900701E090080131
:105AF000F090090120EAC21626E8D20621E0E2066B
:105B0000F104D8F4C701B60122E03DE040E050E0E6
:105B1000AFD0672B682B692B81F485B192E0892780
:105B200085B98BB198E089278BB98BB190E2892731
:105B30008BB985B191E0892785B980EAC81686E8D6
:105B4000D80681E0E806F10428F0109203011092D3
:105B5000020181DDE0900201F090030187011695BA
:105B60000795023192E0190708F05BC0E0FE16C00D
:105B700005DE29873A874B875C876D877E878F870D
:105B8000988B88E0FE013996DE01119601900D9206
:105B90008A95E1F7EFEFEE1AFE0A3BC080910A0109
:105BA000F4E08F9FC00111248233910510F482E349
:105BB00090E04AE0489F9001499F300D112444270E
:105BC00037FD4095542F6091060170910701809137
:105BD0000801909109014CD0672B682B692B41F586
:105BE000F801E55BFE4A849156DD29873A874B87A9
:105BF0005C876D877E878F87988B88E0FE0139965A
:105C0000DE01119601900D928A95E1F72FEFE21ACD
:105C1000F20AF0920301E0920201CE010196F5DC56
:105C200007C04E9905C0109203011092020113DDC6
:105C30008091060190910701A0910801B09109019E
:105C40000196A11DB11DB7FF04C0B695A795979504
:105C500087958093060190930701A0930801B09364
:105C600009018FE891E00197F1F700C00000EACD4B
:105C7000A1E21A2EAA1BBB1BFD010DC0AA1FBB1F50
:105C8000EE1FFF1FA217B307E407F50720F0A21BC2
:105C9000B30BE40BF50B661F771F881F991F1A942F
:105CA00069F760957095809590959B01AC01BD0159
:105CB000CF010895F894FFCFFF5AFFFFFF00221F86
:105CC0001DC010E021C04AE502C032ED432FC4E1FF
:105CD000D0E032E01AB114685F9A0BB11AB954E8F7
:105CE00020E865E320FF05270BB9279517951C3F92
:105CF000F0F66695B8F7B1F720FF05270BB92795A1
:105D000017951C3FD0F62795179517FF052700001C
:105D10001C3F0BB9B0F629913A9519F70B77109102
:105D20002501110FC651D0400BB911F010931F017E
:105D300011E01CBB00681AB11B77402F4B7754E071
:105D40005A95F1F70BB91AB94BB97FCFDC0113960D
:105D50003C911397932F1496EC9114978E2F1296D3
:105D60002C911297203331F4E370F0E0EE5FFE4F98
:105D700080810895283529F4332351F4E1E0F0E0DF
:105D800010C0203599F4332341F4E0E0F0E009C07D
:105D9000383021F5E3E0F0E004C03830F9F4E2E017
:105DA000F0E089E08093570084910895203221F437
:105DB000FC01EE0FFF1F06C0283231F4FC01EE0F8C
:105DC000FF1F319684910895203A09F42BC2203C9C
:105DD00029F415966C912ED280E0089580E0089504
:105DE0001AB880E48BB914BE81E085BF82E085BF1C
:105DF0004E990AC284B7877F84BF88E10FB6F894B2
:105E000080936000109260000FBE809169008260F4
:105E100080936900E89A579A8FEF91EBACE081503C
:105E20009040A040E1F700C000005798789420917E
:105E30002401235027FD54C1309121018CE090E0D2
:105E4000831B91098C01085D1E4F309120013D326A
:105E500009F0C9C0283009F041C123EC2093140196
:105E60002AE52093010110920801D8014C91242FBA
:105E7000207611963C9111972223D1F189E091E08F
:105E80009093230180932201333031F4C8015EDF07
:105E900080930C0124E098C0353031F13A3021F183
:105EA000832F84508630B0F4F801828193819093DF
:105EB0000E0180930D013930C9F0268120930F0126
:105EC00085818270809310013093110147FD78C065
:105ED0002FEF76C080910001323011F48E7F01C027
:105EE00081608093000102C021E06EC020E06CC0A0
:105EF000D80112962C91129710921D01332331F480
:105F000010921E018DE191E022E055C0353019F468
:105F10002093250144C03630E1F5FC01E65DFE4FDB
:105F20002081855D9E4FFC018081813019F48EE1D6
:105F300098E704C0823041F48CE098E79093230105
:105F40008093220122E121C08330F1F4222341F425
:105F50008AE598E7909323018093220124E015C0FD
:105F6000213041F48EE398E790932301809322013E
:105F70002CE10BC0223041F480E398E79093230199
:105F8000809322012EE001C020E080E4809308018C
:105F90001BC0383069F0393029F4209327018DE196
:105FA00091E004C08DE191E03A3021F020E003C09F
:105FB00087E291E021E0909323018093220104C0C5
:105FC00080E8809308010CC0D80117968C91179730
:105FD000882331F416968C911697821708F4282F8F
:105FE000209306017BC08091080187FF77C08091D4
:105FF0000F01E22E821708F4E82E8E1980930F010C
:10600000D1E08111D0E0C0E062C020911101809107
:106010000D0190910E01273068F09C012F5F3F4FDA
:1060200030930E0120930D01F80161918F0102D18F
:10603000CF5F4DC0F0E780309F0708F04DC0CE5FC6
:10604000F894E0910D01F0910E01D8018D919D9190
:106050008D0121E00C0120935700E89511247894DC
:1060600080910D0190910E01029690930E01809304
:106070000D018F779070009741F0DD2341F1CE152F
:1060800030F180911001882311F1F894E0910D0115
:10609000F0910E01329783E080935700E895789451
:1060A00007B600FCFDCFF894E0910D01F0910E01D0
:1060B000329785E080935700E895789407B600FC06
:1060C000FDCFF89481E180935700E8957894CE1540
:1060D00008F49BCFDD2311F01092060110922401E9
:1060E0008091010184FF6CC0809106018F3F09F40B
:1060F00067C0182F893008F018E0811B80930601D3
:106100008091140198E8892780931401112309F4E0
:1061100046C08091080187FF26C080910F0181173A
:1061200008F4182F811B80930F0100E0C5E1D1E036
:1061300017C080911101E0900D01F0900E018730A1
:1061400018F0C7016FD002C0F701849188832196AF
:106150000894E11CF11CF0920E01E0920D010F5F1A
:10616000011739F71AC0E0912201F091230186FF4F
:1061700009C0812FA5E1B1E094919D9331968150A2
:10618000D9F707C0812FA5E1B1E091919D9381508E
:10619000E1F7F0932301E0932201193058F485E1EF
:1061A00091E0612FBBDC1C5F1C3041F08FEF8093CE
:1061B000060104C08FEF809306011EE110930101D8
:1061C00084E199B1947831F48150D9F71092250186
:1061D00010921F0180910001803130F04E9B0FC062
:1061E00080910001805109C04E9909C08091000141
:1061F000823028F0809100018250809300018091CC
:106200000001882309F013CEF894579A1BB81DBAE1
:106210001092690081E085BF15BEE0911201F091F6
:1062200013010995F999FECF92BD81BDF89A99277E
:1062300080B50895262FF999FECF1FBA92BD81BD72
:1062400020BD0FB6F894FA9AF99A0FBE01960895F8
:10625000F894FFCFFE5A1E950F00FF00FA01DC01F3
:1062600002C005900D9221503040D8F70895AF92AA
:10627000BF92CF92DF92EF92FF920F931F93CF9333
:10628000DF93CDB7DEB7C058D0400FB6F894DEBF6D
:106290000FBECDBF88E10FB6F894809360001092D6
:1062A00060000FBEF89488E28AB983E084B980E286
:1062B0008BB91982609100017091010120E030E0FA
:1062C000FB01E20FF31F45915491F901E050F049B1
:1062D000859194914817590719F081E0898306C088
:1062E0002E5F3F4F80E12030380751F789818823A6
:1062F00009F499C078E6C72E70E7D72EE12CF12C6F
:10630000C701B601AE014F5F5F4F20E830E00E9449
:106310009E289C01C701B6016856724F8F4F9F4F50
:10632000AE014F5F5F4F02E518E20E94B42880E89B
:1063300090E0A0E0B0E0C80ED91EEA1EFB1E98E671
:10634000C91692E7D90690E0E90690E0F906C1F691
:10635000C12C60E7D62EE12CF12CA12C50E9B52EF2
:10636000AC0CBD1C40910001509101014A0D5B1D18
:10637000662757FD6095762FCE01019620E830E024
:106380006DDFC701B601AE014F5F5F4F20E830E01F
:1063900008E718E20E94B42880E890E0A0E0B0E0AE
:1063A000C80ED91EEA1EFB1E90E0C91693E7D90657
:1063B00090E0E90690E0F90681F6C12C40E1D42E88
:1063C000CA18DB0840910001509101014A0D5B1D84
:1063D000662757FD6095762F9601A1E8CA16D1046D
:1063E00010F020E830E0CE01019638DFB5016050B2
:1063F000704980E090E0AE014F5F5F4F20E830E0F1
:1064000002E518E20E94B42880E890E0A80EB91EC8
:10641000A0E8BFEFCA0EDB1EB0E0AB16B0E1BB06D2
:1064200088F282E085B9289AC058DF4F0FB6F894F9
:10643000DEBF0FBECDBFDF91CF911F910F91FF90B7
:10644000EF90DF90CF90BF90AF900895F894FFCF7A
:106450005C52FFFFFFFFFFFFFFFFFFFFFFFFFFFF9C
:10646000FFFFFFFFFFFFFFFFFFFFFFFFFFFFFFFF3C
:10647000FFFFFFFFFFFFFFFFFFFFFFFFFFFFFFFF2C
:10648000FFFFFFFFFFFFFFFFFFFFFFFFFFFFFFFF1C
:10649000FFFFFFFFFFFFFFFFFFFFFFFFFFFFFFFF0C
:107000000FC400005EC4000032C4000030C40000A1
:107010002EC400002CC400002AC4000028C40000B4
:1070200026C4000024C4000022C4000020C40000C4
:107030001EC400001CC400001AC4000018C40000D4
:1070400016C4000014C4000012C4000010C40000E4
:107050000EC400000CC400000AC4000008C40000F4
:1070600006C4000004C400007E3FF9F76A39F9F74E
:107070005635F9F74038F9F7EC2DFD2DB7B6B0FCD1
:10708000FDCF27BFE895B7B6B0FCFDCF21E1B7B67D
:10709000B6FCF4CF0895FFFFFFFFFFFFFFFFFFFFE8
:1070A000FFFFFFFFFFFFFFFFFFFFFFFFFFFFFFFFF0
:1070B000FFFFFFFFFFFFFFFFFFFFFFFFFFFFFFFFE0
:1070C000FFFFFFFFFFFFFFFFFFFFFFFFFFFFFFFFD0
:1070D000FFFFFFFFFFFFFFFFFFFFFFFFFFFFFFFFC0
:10779000FFFF5553426173704C6F616465722076D0
:1077A000302E39372C206279205374657068616EF1
:1077B0002042616572776F6C6620286D6174726912
:1077C0007873746F726D40676D782E646529090255
:1077D00012000101008032090400000000000000D6
:1077E00012011001FF000008C016DC0502010102B1
:1077F00000010E0355005300420061007300700049
:107800001C037700770077002E0066006900730084
:10781000630068006C002E00640065000403090426
:1078200011241FBECFEFD8E0DEBFCDBF24B7D8E014
:10783000CEEF39913833399109F03FEF30933E0163
:1078400020933D0111E0A0E0B1E0EAEFFFE702C0C4
:1078500005900D92A630B107D9F721E0A6E0B1E07E
:1078600001C01D92AD33B207E1F787D1C4C3C8CBC5
:10787000A82FB92F8FEF9FEF1BC02D918227282FA4
:1078800022952827722F269526952727239526951A
:107890002170782F892F82272195207C922F2227F3
:1078A000769527959727822776952795972782277C
:1078B000615018F7809590950895DADF8D939D9328
:1078C0000895CF93CFB7CF93DF93C3954F9BE9F73D
:1078D0004F9B0BC04F9B09C04F9B07C04F9B05C0E0
:1078E0004F9B03C04F9B01C089C06F93C091200183
:1078F000DD27C95DDE4F2F9365E54F9B03C02F91B8
:107900006F91E6CF0F931F934F9320E040E15F9379
:1079100009B1047807FB27F93F9350E03BE039C0F9
:10792000147840642F77012F5F5F1EC0406819B143
:1079300014782F7752501FC0406409B12F77047814
:10794000D1F15F5F00C023C0406219B12F77147876
:1079500091F15F5F00C025C004781027515012F4E8
:107960005D5F0000115027952C3F19B1C8F61478BF
:107970000127015027952C3FC8F64227499309B1AA
:10798000047810274F73115027952C3FA8F6469581
:10799000469519B1147879F00127015027952C3FAD
:1079A00098F66B5A60F3315009B1B0F600C011E09F
:1079B0001CBB002717C03B503195C31BD04011E0C2
:1079C0001CBB0881033CF9F00B34E9F020911E0147
:1079D0001981110F1213EDCF093651F10D3211F04B
:1079E000013E39F7009325013F915F914F911F911F
:1079F0000F912F916F91CCB3C0FD67CFDF91CF91E5
:107A0000CFBFCF91189520912501222369F31091C2
:107A10002301112339F534303AF1309323012093B7
:107A20001F01109120013BE0311B309320011CC04D
:107A3000009123010130B4F40AE53091010134FDD5
:107A400014C000930101C3E1D1E013C0052710E089
:107A500000C000000BB91AC0052710E0221F1DC08E
:107A600010E021C04AE502C032ED432FC4E1D0E06E
:107A700032E01AB114685F9A0BB11AB954E820E8E1
:107A800065E320FF05270BB9279517951C3FF0F6F6
:107A90006695B8F7B1F720FF05270BB9279517951D
:107AA0001C3FD0F62795179517FF052700001C3FB0
:107AB0000BB9B0F629913A9519F70B77109124017B
:107AC000110FC651D0400BB911F010931E0111E0F7
:107AD0001CBB00681AB11B77402F4B7754E05A95B6
:107AE000F1F70BB91AB94BB97FCFFC013381932F52
:107AF0004481842F2281203339F44370E42FF0E055
:107B0000EE5FFE4F80810895283529F431110EC0B3
:107B1000E1E0F0E006C0203599F431110CC0E0E05E
:107B2000F0E089E08093570084910895383019F58A
:107B3000E3E0F0E0F6CF3830F1F4E2E0F0E0F1CF4E
:107B4000203221F4FC01EE0FFF1F06C0283231F471
:107B5000FC01EE0FFF1F319684910895203A09F43D
:107B600034C2203C19F4658138D205C02F3F19F486
:107B700081EF8093110180E008951AB880E48BB9F9
:107B800081E085BF82E085BF2FEF80E792E0215042
:107B900080409040E1F700C0000080913D01877F68
:107BA00021F480913E01882381F04E9B0EC0F89411
:107BB000579A1BB81DBA1092690081E085BF15BEA7
:107BC000E0910A01F0910B0109958EEF809311016C
:107BD00084B7877F84BF88E10FB6F89480936000F4
:107BE000109260000FBE14BE809169008260809385
:107BF0006900E89A579AEFEFF1EB2CE0E150F04082
:107C00002040E1F700C0000057987894809123014C
:107C1000835087FD46C190912001CCE0D0E0C91B84
:107C2000D109C95DDE4F90911F019D3209F0B9C0A5
:107C3000883009F034C183EC809313018AE5809386
:107C40000101109212014881842F807639818823A6
:107C5000B9F186E091E090932201809321013330C5
:107C600031F4CE0142DF8093090124E090C0353029
:107C700019F13A3009F18CEF830F863098F48A813C
:107C80009B819093100180930F013930B9F08E8160
:107C900080930E018D81827080930D0130930C01D1
:107CA0002FEF6FC080911101323011F48E7F01C02F
:107CB00081608093110102C021E069C020E067C0AB
:107CC0008A8110921C01311106C010921D018CE1B5
:107CD00091E022E050C0353019F4809324013DC07A
:107CE0003630A9F59B81913019F480EE97E704C0F6
:107CF000923041F48EEC97E790932201809321011A
:107D000022E121C09330F1F4811108C08CE198E7A1
:107D1000909322018093210124E015C0813041F429
:107D200080E098E790932201809321012CE10BC021
:107D3000823041F482EF97E79093220180932101F2
:107D40002EE001C020E080E48093120118C038309A
:107D500079F0393031F4809326018CE191E020E014
:107D60000AC021E03A3009F020E08CE191E003C044
:107D700086E291E021E090932201809321012F3F40
:107D800031F447FD2E8180E88093120107C08F8176
:107D9000811104C08E81821708F4282F20930001DE
:107DA0007EC09091120197FF7AC090910E01E82E4B
:107DB000981708F4E92E9E1990930E01DD24D394B0
:107DC0009111D12CF12CFE1408F066C020910C0109
:107DD00080910F0190911001273078F08E010F5F94
:107DE0001F4F68819C012F5F3F4F309310012093FC
:107DF0000F01F3D0F394E801E6CF8115904708F026
:107E00004CC0F394F394F894E0910F01F0911001B9
:107E10008991999121E00C0120935700E895112454
:107E2000789480910F019091100102969093100127
:107E300080930F018F779927892B59F0DD2009F462
:107E4000C2CFFE1408F4BFCF80910D01882309F43E
:107E5000BACFF894E0910F01F0911001329783E0CE
:107E600080935700E895789407B600FCFDCFF8940E
:107E7000E0910F01F0911001329785E08093570057
:107E8000E895789407B600FCFDCFF89481E18093E3
:107E90005700E895789497CFD11010920001109276
:107EA00023018091010184FF6CC0809100018F3F0C
:107EB00009F467C0F82E893010F028E0F22E8F19EF
:107EC000809300018091130198E889278093130122
:107ED000FF2009F449C08091120187FF27C08091DB
:107EE0000E018F1508F4F82E8F1980930E01E09083
:107EF0000C01C4E1D1E084E191E0FC2FF81BFF15F7
:107F000098F500910F0110911001F6E0FE1518F49C
:107F1000C8015BD002C0F8018491888321960F5F6D
:107F20001F4F1093100100930F01E5CFE091210145
:107F3000F091220186FF0BC084E191E0DC012491E5
:107F40002D9331962F2D280F2A13F9CF09C084E1E4
:107F500091E0DC0121912D932F2D280F2A13FACFC8
:107F6000F0932201E09321016F2D84E191E0A5DCE3
:107F700084E08F0D8C3019F09FEF90930001809377
:107F8000010184E199B1947831F48150D9F71092CC
:107F9000240110921E0180911101803130F04E9B1E
:107FA0000FC080911101805109C04E9909C0809184
:107FB0001101823028F080911101825080931101CB
:107FC00080911101811122CEF2CDF999FECF92BD9F
:107FD00081BDF89A992780B50895262FF999FECF8B
:107FE0001FBA92BD81BD20BD0FB6F894FA9AF99AD6
:107FF0000FBE01960895F894FFCFFF5A1E950F000B
:00000001FF
